:020000040800F2
:10000000A80C002049010008A5150008A715000844
:10001000AB150008AF150008B3150008000000007C
:10002000000000000000000000000000B7150008FC
:10003000B915000800000000BB150008BD15000838
:100040006301000863010008630100086301000800
:1000500063010008630100086301000863010008F0
:1000600063010008630100086301000863010008E0
:1000700063010008630100086301000863010008D0
:1000800063010008630100086301000863010008C0
:1000900063010008630100086301000863010008B0
:1000A00063010008630100086301000863010008A0
:1000B0006301000863010008630100086301000890
:1000C0006301000863010008630100086301000880
:1000D000630100084316000863010008FB160008CE
:1000E0006301000863010008630100086301000860
:1000F0006301000863010008630100086301000850
:10010000630100086301000863010008630100083F
:10011000630100086301000863010008630100082F
:10012000630100086301000863010008630100081F
:10013000DFF810D003F0CAFF004800475D10000848
:10014000AFF30080A80C002006488047064800470F
:10015000FEE7FEE7FEE7FEE7FEE7FEE7FEE7FEE777
:10016000FEE7FEE74B020008310100080CB5002055
:10017000019000906C48006840F480306A49086043
:1001800000BF6948006800F4003000900198401CEE
:100190000190009818B90198B0F5A06FF1D16248AC
:1001A000006800F4003010B10120009001E0002050
:1001B00000900098012843D15C48006840F010008E
:1001C0005A4908600846006820F0030008600846A5
:1001D000006840F002000860534840685249486097
:1001E0000846406848600846406840F480604860BF
:1001F0000846406820F47C1048600846406840F497
:10020000E81048600846006840F08070086000BF51
:100210004548006800F000700028F9D04248406866
:1002200020F00300404948600846406840F0020062
:10023000486000BF3C48406800F00C000828F9D135
:100240000CBD10B5FFF792FF10BD10B53648006821
:1002500040F00100344908600846406834490840CD
:100260003149486008460068324908402E49086014
:100270000846006820F4802008600846406820F4A2
:10028000FE0048604FF41F008860FFF7DAFF4FF070
:1002900000602949086010BD10B50021002000222F
:1002A000214B5B6803F00C0121B1042906D0082919
:1002B00028D107E0214B224C236027E01F4B204C24
:1002C000236023E0184B5B6803F47010164B5B68E7
:1002D00003F48032022303EB904022B9194B4343CD
:1002E000174C23600DE0104B5B6803F4003323B11F
:1002F000144B4343124C236003E0104B4343104C18
:10030000236003E00D4B0E4C236000BF00BF064B83
:100310005B68C3F303130C4CE15C094B1B68CB40D7
:10032000074C236010BD0000001002400020024076
:100330000000FFF8FFFFF6FE08ED00E000127A0073
:100340000000002000093D00040000203149014365
:10035000314A1160704770B5002100230F22C47824
:1003600004B32D4C246804F4E064C4F5E064210A6D
:10037000C1F10403CA40447804FA03F184781440BC
:1003800021430901254C0678A155047804F01F0586
:100390000124AC4005786D11AD0005F1E025C5F8EC
:1003A000004109E0047804F01F050124AC401C4D15
:1003B0000678761145F8264070BD1A4A0A40024375
:1003C000154B1B1F1A60704739B1134A121D126872
:1003D0000243114B1B1D1A6006E00F4A121D1268E2
:1003E00082430D4B1B1D1A607047042808D14FF043
:1003F000E021096941F004014FF0E022116107E0BA
:100400004FF0E021096921F004014FF0E022116171
:10041000704700000000FA050CED00E000E400E089
:1004200080E100E080FFFF1F10B50446CC48844205
:1004300008D10121042000F04DFB0021042000F030
:1004400049FB46E0C748844208D10121082000F05A
:1004500041FB0021082000F03DFB3AE0C248844205
:1004600008D10121102000F035FB0021102000F000
:1004700031FB2EE0BD48844208D10121202000F04C
:1004800029FB0021202000F025FB22E0B84884420F
:1004900008D10121402000F01DFB0021402000F088
:1004A00019FB16E0B348844208D10121802000F0F6
:1004B00011FB0021802000F00DFB0AE0AE488442D1
:1004C00007D10121801500F005FB0021A01500F0E7
:1004D00001FB10BD10B50121084600F0FBFA002118
:1004E000012000F0F7FA10BD2DE9F0410246002589
:1004F0000026002000230024002791F803C00CF000
:100500000F0591F803C00CF0100CBCF1000F03D0E4
:1005100091F802C04CEA050591F800C0BCF1000F4B
:1005200031D0146800202BE04FF0010C0CFA00F3DE
:10053000B1F800C00CEA03069E4220D183004FF0C0
:100540000F0C0CFA03F7BC4305FA03FC4CEA040455
:1005500091F803C0BCF1280F06D14FF0010C0CFA42
:1005600000FCC2F814C00AE091F803C0BCF1480FC7
:1005700005D14FF0010C0CFA00FCC2F810C0401C71
:100580000828D1D31460B1F800C0BCF1FF0F34DDEE
:10059000546800202EE000F1080C4FF0010808FA22
:1005A0000CF3B1F800C00CEA03069E4221D183008F
:1005B0004FF00F0C0CFA03F7BC4305FA03FC4CEAAE
:1005C000040491F803C0BCF1280F05D100F1080C18
:1005D00008FA0CF8C2F8148091F803C0BCF1480F77
:1005E00007D100F1080C4FF0010808FA0CF8C2F826
:1005F0001080401C0828CED35460BDE8F0814FF62F
:10060000FF710180022181700421C1707047024690
:10061000002093680B400BB1012000E000207047E0
:100620000146886880B2704702460020D3680B40BC
:100630000BB1012000E0002070470146C86880B27D
:10064000704701617047416170470AB1016100E084
:1006500041617047C16070474FF480320A43826144
:100660008161826182698269704702460020434B42
:1006700018684FF68073184040EA021008433F4B59
:10068000186070473E49C8617047F0B50A460023BC
:1006900000240021002500F00046B6F1004F02D1F1
:1006A000364EF16901E0354E7168C0F3034583B2FF
:1006B00000F44016B6F5401F08D121F070612F4EAE
:1006C000766826F070662D4F7E6012E000F480168A
:1006D000B6F5801F06D1032606FA05F4A14341F0C2
:1006E000706106E0460D360103FA06F6B14341F0AB
:1006F000706122B1460D360103FA06F6314300F06F
:100700000046B6F1004F02D11C4EF16101E01B4ED4
:100710007160F0BD30B500228B071C0F0F2303FA68
:1007200004F2164B08338C1053F824309343134CC7
:1007300008348D1044F8253023468C1053F82430AB
:100740008C07240F00FA04F423430C4C08348D105A
:1007500044F8253030BD0A49DC310860704700009C
:1007600000080140000C014000100140001401404D
:1007700000180140001C0140002001400000014021
:10078000000020420E49086070470D4948607047DC
:100790000B49886070474AF6AA20094908607047EB
:1007A0004CF6CC4006490860704701460020044AD8
:1007B000D2680A400AB1012000E000207047000022
:1007C00000300040DF48006840F00100DD4908606B
:1007D00008464068DC490840DA4948600846006835
:1007E000DA490840D74908600846006820F48020AC
:1007F00008600846406820F4FE0048604FF41F007F
:1008000088607047CF49096821F48031CD4A116072
:100810001146096821F480211160B0F5803F03D0B2
:10082000B0F5802F0ED106E0C649096841F4803149
:10083000C44A116007E0C349096841F4A021C14AD4
:10084000116000E000BF00BF704710B501460022F4
:10085000002300204A11012A02D1BA4C236806E085
:10086000022A02D1B74C236A01E0B64C636A01F058
:100870001F02012494401C400CB1012000E0002024
:1008800010BD38B5002000900024002500BF3120A5
:10089000FFF7DBFF05460098401C00900098B0F57C
:1008A000A06F01D0002DF2D03120FFF7CEFF08B1AC
:1008B000012400E00024204638BD01460020A14A62
:1008C000106820F0F80040EAC10010607047A049AD
:1008D00008607047024600209A4B586820F47C104C
:1008E00042EA01031843974B5860704798490866DD
:1008F000704701460020934A506820F003000843E7
:10090000506070478F48406800F00C007047014607
:1009100000208C4A506820F0F00008435060704777
:1009200001460020874A506820F4E0600843506088
:10093000704701460020834A506820F4605040EA26
:10094000C1005060704729B17E4A527A02437D4B04
:100950005A7204E07B4A527A82437A4B5A72704749
:100960007B49D8310860704701460020754A5068BD
:1009700020F440400843506070470021714A203203
:100980001170704A82F82010012802D004280AD180
:1009900004E001216B4A2032117005E00521694A0B
:1009A0002032117000E000BF00BF70476949086045
:1009B00070476449096A0143624A11627047654998
:1009C00044390860704730B500210022002400231C
:1009D0005C4D6D6805F00C0121B1042905D0082992
:1009E00023D105E05C4D056022E05B4D05601FE012
:1009F000544D6D6805F47012524D6D6805F48034E5
:100A0000022505EB92421CB9544D554305600BE09D
:100A10004C4D6D6805F400351DB1504D55430560D2
:100A200002E04D4D5543056002E04B4D056000BFAF
:100A300000BF444D6D6805F0F0010909484D6B5C3D
:100A40000568DD4045603F4D6D6805F4E061090AC9
:100A5000434D6B5C4568DD4085603A4D6D6805F43B
:100A60006051C90A3E4D6B5C4568DD40C560354D3F
:100A70006D6805F44041890B3A4D6B5CC568B5FB68
:100A8000F3F5056130BD29B12E4A526902432D4B61
:100A90005A6104E02B4A526982432A4B5A617047DB
:100AA00029B1284A92690243264B9A6104E0254AFB
:100AB00092698243234B9A61704729B1214AD269D6
:100AC0000243204BDA6104E01E4AD26982431D4B87
:100AD000DA61704729B11B4AD2680243194BDA60C8
:100AE00004E0184AD2688243164BDA60704729B195
:100AF000144A12690243134B1A6104E0114A126945
:100B00008243104B1A6170471249403908607047A0
:100B10000F49C86470470B49C87170470948406A5B
:100B200040F0807007494862704701460020054A3E
:100B300092680A400AB1012000E000207047014994
:100B400088727047001002400000FFF8FFFFF6FEB9
:100B5000000042428004424200127A0000093D0037
:100B6000140000202400002010B50446FB488442F5
:100B700009D101218803FFF7ADFF00214FF4804028
:100B8000FFF7A8FF32E0F648844209D1012148046A
:100B9000FFF7ADFF00214FF40030FFF7A8FF25E07D
:100BA000F048844209D101218804FFF7A0FF002109
:100BB0004FF48020FFF79BFF18E0EB48844209D1F7
:100BC0000121C804FFF793FF00214FF40020FFF735
:100BD0008EFF0BE0E548844208D101210805FFF7AC
:100BE00086FF00214FF48010FFF781FF10BD2DE933
:100BF000F04786B005460E460024A24600BFA14637
:100C00000027B08900B100BF2F462C8A4CF6FF7038
:100C10000440F08804432C82AC894EF6F310044063
:100C2000B08831890843718908430443AC81AC8A98
:100C30004FF6FF400440B0890443AC8201A8FFF79F
:100C4000C2FEC648874202D1DDF810A001E0DDF8FF
:100C50000CA0A88900F4004040B10AEBCA0000EBE8
:100C60000A1031684900B0FBF1F807E00AEBCA004E
:100C700000EB0A1031688900B0FBF1F86420B8FB82
:100C8000F0F004012009642101FB1089A88900F417
:100C9000004040B1322000EBC900B0FBF1F000F0A1
:100CA0000700044308E0322000EB09106421B0FB88
:100CB000F1F000F00F0004432C8106B0BDE8F0878E
:100CC0004FF41651016000218180C18001810C2107
:100CD000418100218181704710B502460020108AB1
:100CE0004FF2FF0318400B884C8823438C88234322
:100CF000CC8823431843108210BD0021018041801D
:100D00008180C180704721B1828942F40052828182
:100D100004E082894DF6FF731A4082817047F0B576
:100D20000346002400260025002040F66A17B94239
:100D300000D100BF1846C1F3421401F01F0601277D
:100D400007FA06F5012C01D10C3004E0022C01D188
:100D5000103000E014301AB107682F43076002E03A
:100D60000768AF430760F0BD1AB1838A0B438382E3
:100D700002E0838A8B4383827047028A4FF6F073C6
:100D80001A400282028A0A430282704782894FF225
:100D9000FF731A40828182890A438281704721B1A0
:100DA000828942F00202828104E082894FF6FD735B
:100DB0001A4082817047028A4FF6DF731A4002821E
:100DC000028A0A430282704721B1028A42F48042B9
:100DD000028204E0028A4BF6FF731A4002827047D7
:100DE000C1F308028280704701468888C0F308007A
:100DF0007047818941F0010181817047028BD2B235
:100E00000283028B42EA012202837047028B02F4C2
:100E10007F420283028B0A430283704721B1828A98
:100E200042F02002828204E0828A4FF6DF731A4089
:100E30008282704721B1828A42F01002828204E0ED
:100E4000828A4FF6EF731A408282704721B1828AFC
:100E500042F00802828204E0828A4FF6F7731A4059
:100E60008282704721B1828942F40042828103E08C
:100E70008289C2F30E028281704721B1828A42F4D4
:100E80000062828204E0828A4FF2FF731A408282FB
:100E90007047828A4FF6FB731A408282828A0A4325
:100EA0008282704721B1828A42F00202828204E08B
:100EB000828A4FF6FD731A408282704702460020F4
:100EC000B1F5007F00D100BF13880B400BB10120AA
:100ED00000E00020704701F40072B2F5007F00D1FD
:100EE00000BFCA430280704770B502460024002349
:100EF0000025002040F66A16B14200D100BFC1F3C0
:100F0000421501F01F03012606FA03F3012D02D159
:100F10009689334006E0022D02D1168A334001E063
:100F2000968A33400C12012606FA04F416883440DF
:100F300013B10CB1012000E0002070BD10B50022FB
:100F4000002340F66A14A14200D100BF0A12012416
:100F50009440A3B2DC43048010BD0000003801407F
:100F60000044004000480040004C00400050004059
:100F70001FB58DA003F0DCF801F0C7FB002854D0AA
:100F8000954801F07FFB00284BD19348016893A05E
:100F900003F0CEF89048C279817995A003F0C8F8A3
:100FA0008D484279017997A003F0C2F88A48017A06
:100FB00099A003F0BDF88848407AAA2801D19BA0E7
:100FC00000E09CA001469DA003F0B2F801F0A1FB57
:100FD000044621469EA003F0ABF801F09EFB08B941
:100FE000A0A000E0A3A004462146A7A003F0A0F81B
:100FF0007948C3798279A9A102A803F0A9F802AAC5
:101000000621012000F080FE734843790279A3A1F4
:10101000684603F09DF86A460621022000F074FE3F
:1010200006E0A0A003F084F802E0A5A003F080F899
:10103000ABA003F07DF81FBD10B57D20FFF705FCC8
:10104000012805D1AFA003F073F8FFF767FD04E0B6
:10105000B1A003F06DF8FFF761FD10BD01F0AFF82E
:10106000FFF7EAFF02F0BCFFAFA003F061F800F069
:1010700079FC00F0F1FC01F06FF800F093FF02F052
:10108000F5F800F0C8FF00F035FFB4A003F050F809
:10109000C14803F04DF8C14803F04AF8C0A003F07E
:1010A00047F8C8A003F044F8D1A003F041F8DC48A9
:1010B00003F03EF802F05FFD00F092FCD9A003F0CF
:1010C00037F801F0B1FA0446002C13D1E0A003F088
:1010D0002FF801F0C0FB01F018FB38B101F019FB4B
:1010E00005462946E4A003F023F80AE074A003F0C3
:1010F0001FF806E02146EAA003F01AF8F5A003F075
:1011000017F800220121084600F012FE05220221F4
:10111000012000F00DFE3A220521012000F0BDFD66
:1011200043220A21012000F0B8FD012211460220CD
:1011300000F0FEFD05220221084600F0F9FD3A22EA
:101140000521022000F0A9FD25220A21022000F03D
:10115000A4FDEFA20121032000F0D6FD44A201214D
:10116000042000F0D1FD03E2FFF715FBEC48006816
:10117000401CEB49086002F0B0FD0121E94800F095
:1011800021FF01280FD100F0FEFF38B11021E54802
:10119000FFF759FAE4A002F0CBFFDCE11021E148AF
:1011A000FFF74FFAD4E1D9E10D0A3D3D3D2057321A
:1011B00035513634E4B8ADE5AD98E582A8E79A84B8
:1011C000E69C80E696B04448543131E695B0E68D11
:1011D000AE203D3D3D0D0A006C000020E697B6E9CB
:1011E00097B4E688B33A202564E7A7925C720A00B8
:1011F000E6B8A9E5BAA63A2025642E2564E28483E0
:101200005C720A00E6B9BFE5BAA63A2025642E252D
:1012100064252552480D0A00E6A0A1E9AA8CE592B2
:101220008C3A203078253032580D0A00E69C89E649
:1012300095880000E697A0E695880000E695B0E660
:101240008DAEE78AB6E680813A2025730D0A00004C
:10125000E680BBE8AEB0E5BD95E695B03A202564E2
:101260000D0A0000E8A686E79B96E6A8A1E5BC8FDC
:1012700000000000E78EAFE5BDA2E7BC93E586B2B3
:10128000E6A8A1E5BC8F0000E5AD98E582A8E6A838
:10129000A1E5BC8F3A2025730D0A00002532642E8B
:1012A00025640000E8AFBBE58F96573235513634E0
:1012B000E695B0E68DAEE5A4B1E8B4A50D0A000050
:1012C000573235513634E4B8ADE69A82E697A0E657
:1012D0009C89E69588E695B0E68DAE5C720A0000C2
:1012E0003D3D3D3D3D3D3D3D3D3D3D3D3D3D3D3D2E
:1012F0003D3D3D3D3D3D3D3D3D3D3D3D3D3D3D3D1E
:101300000D0A00005741544348444F475F5245532C
:1013100045540D0A000000004E4F524D414C5F52A3
:10132000455345540D0A0000E79C8BE997A8E78BCD
:1013300097E5889DE5A78BE58C96E5AE8CE68890D1
:10134000EFBC8CE8B685E697B6E697B6E997B4E7C2
:10135000BAA63230E7A7925C720A00000D0A57461F
:101360002D455350383236362057694669E6A8A1D4
:10137000E59D97E7BBBCE59088E6B58BE8AF95E7C0
:10138000A88BE5BA8F202D20573235513634E789A6
:1013900088E69CAC0D0A00006C4E0008F04E000878
:1013A0000D0AE694AFE68C81E79A844C4544E68EBC
:1013B000A7E588B6E591BDE4BBA4EFBC9A5C720AD0
:1013C000000000004C45445F5245442C204C4544ED
:1013D0005F475245454E2C204C45445F424C554595
:1013E0002C204C45445F59454C4C4F570D0A00008A
:1013F0004C45445F505552504C452C204C45445F61
:101400004359414E2C204C45445F57484954452C84
:10141000204C45445F5247424F46460D0A000000AB
:10142000284E00080D0AE6ADA3E59CA8E5889DE5D9
:10143000A78BE58C96573235513634E5AD98E58269
:10144000A8E7B3BBE7BB9F2E2E2E0D0A00000000BD
:10145000573235513634E5AD98E582A8E7B3BBE79E
:10146000BB9FE5889DE5A78BE58C96E68890E58A8D
:101470009FEFBC810D0A0000E58F91E78EB0E78EEB
:10148000B0E69C89E695B0E68DAEEFBC8CE680BBFD
:10149000E8AEB0E5BD95E695B03A2025640D0A00AA
:1014A000573235513634E5AD98E582A8E7B3BBE74E
:1014B000BB9FE5889DE5A78BE58C96E5A4B1E8B4D4
:1014C000A5EFBC81E99499E8AFAFE7A0813A202568
:1014D000640D0A00E7A88BE5BA8FE5B086E7BBA7E5
:1014E000E7BBADE8BF90E8A18CEFBC8CE4BD86E41F
:1014F000B88DE4BC9AE4BF9DE5AD98E695B0E68D65
:10150000AEE588B05732355136340D0A0000000080
:101510005732355136345F444154413A000000009F
:1015200028000020000801400D0AE68C89E994AEED
:10153000E68C89E4B88BEFBC9AE7BBA7E794B5E5E6
:1015400099A8E5B7B2E585B3E997AD5C720A0000EA
:1015500008A002F0EDFD114800F016FA10480068EE
:1015600030B102F061FB00200D490860FFF700FD7B
:10157000FAE500000D0AE68C89E994AEE68C89E470
:10158000B88BEFBC9AE7BBA7E794B5E599A8E5B798
:10159000B2E68993E5BC800D0A000000400D03000F
:1015A00034000020704700BFFEE700BFFEE700BF29
:1015B000FEE700BFFEE770477047704770B5002434
:1015C00007E0814850F82400401C7F4941F824007E
:1015D000641C022CF5DB7D480088401C7B49088098
:1015E00008460088642806DB0020088078480068E8
:1015F000401C7749086074480068C82819D3002047
:10160000714908607348006898B9734800F053FD49
:1016100001280AD16F4908606D4801686E4801F0E1
:1016200017F8054605B100BF03E04FF0FF306949E8
:10163000086065484068322802D30020624948604B
:1016400070BD10B540F225516448FFF74DFCD8B18C
:101650006248FFF7C9FBC4B26148B0F80004C0F3A8
:101660000E0040F2FF3188420EDA5D49B1F80014F5
:10167000C1F30E00411C5A4AB2F8002461F30E0275
:101680005749A1F800240C5440F224415348FFF775
:101690002BFC012830D15248B0F8000420F400405F
:1016A00000F500404E49A1F8000420214B48FFF707
:1016B00005FC01281CD14948FFF796FBC4B24848F5
:1016C000B0F80004C0F30E0040F2FF31884213DA94
:1016D0004349B1F80014C1F30E00411C404AB2F86E
:1016E000002461F30E023E49A1F800240C5403E0EB
:1016F0003A48FFF779FBC4B210BD10B540F225514E
:101700003848FFF7F1FBD8B13648FFF76DFBC4B29C
:101710003548B0F80004C0F30E0040F2FF318842B3
:101720000EDA3149B1F80014C1F30E00411C2E4A03
:10173000B2F8002461F30E022B49A1F800240C54E6
:1017400040F224412748FFF7CFFB01283AD1264831
:10175000B0F8000420F4004000F500402249A1F850
:10176000000420211F48FFF7A9FB01281CD11D48B8
:10177000FFF73AFBC4B21C48B0F80004C0F30E00F7
:1017800040F2FF31884213DA1749B1F80014C1F36F
:101790000E00411C144AB2F8002461F30E021249F3
:1017A000A1F800240C5403E00E48FFF71DFBC4B25F
:1017B0000EA10D4802F040FC08B1012000E000201D
:1017C0000D49087010BD00002C0000203C000020D6
:1017D0003800002034000020600000200038014064
:1017E000A204002000480040A0000020434C4F53BA
:1017F00045440D0A0000000065000020F0B50346D6
:101800000D461646002729460A2E03D000200870F0
:101810002846F0BD33B9302001F8010B00200870D4
:101820002846F6E7002B03DA2D2001F8010B5B4276
:1018300042F210720DE093FBF2F404B937B104F1F7
:10184000300001F8010B04FB123301270A2092FB40
:10185000F0F2002AEFDC002008702846D9E70FB428
:1018600070B586B006460CA8019073E00B9800781E
:101870005C281CD10B98401C0B9000786E2809D076
:1018800072280FD10D213046FFF7AAFA0B98401CA1
:101890000B900BE00A213046FFF7A2FA0B98401C90
:1018A0000B9003E00B98401C0B9000BF4BE00B9893
:1018B0000078252840D10B98401C0B9000786428B4
:1018C00018D0732833D1019810C801900BE021780B
:1018D0003046FFF785FA00BF80213046FFF7EEFA69
:1018E0000028F9D0641C20780028F0D10B98401C07
:1018F0000B9020E0019820C801900A2202A92846F6
:10190000FFF77CFF02AC0BE021783046FFF768FA66
:1019100000BF80213046FFF7D1FA0028F9D0641CBF
:1019200020780028F0D10B98401C0B9003E00B9816
:10193000401C0B9000BF06E00B9810F8011B0B90A9
:101940003046FFF74DFA00BF80213046FFF7B6FA68
:101950000028F9D00B980078002887D106B070BC19
:101960005DF814FB1A48006840F080701849086060
:101970000020184948600846006840F001000860EF
:10198000704714484068704731B50023124800681A
:10199000124DB0FBF5F0009D00FB05F400BFFFF712
:1019A000F0FF024611E0FFF7ECFF014691420CD038
:1019B000914202D9881A034403E0C2F1FF3008447F
:1019C00003440A46A34200D300E0ECE700BF38BD61
:1019D000FCED00E0001000E00000002040420F009D
:1019E00030B51A4800686422B0FBF2F1B1F1807F93
:1019F00001D301201DE021F07F40401E4FF0E02286
:101A0000506150170F22002807DA13071D0E104BE4
:101A100000F00F04241F1D5503E013071C0E0D4B8F
:101A20001C5400BF00204FF0E0229061072010619D
:101A3000002008B100BFFEE74FF0E020006940F051
:101A400001004FF0E021086130BD000000000020DF
:101A500018ED00E000E400E008B501210820FFF7E0
:101A60001FF82020ADF8000010208DF8030003209F
:101A70008DF8020069461148FEF736FD0120ADF8E9
:101A8000000069460D48FEF72FFD0220ADF800006A
:101A900069460A48FEF728FD20210848FEF7D1FDD7
:101AA00001210648FEF7CDFD02210448FEF7C9FDDD
:101AB00008BD2022014B14331A607047000C01400E
:101AC00008B501210820FEF7EBFF14208DF8030074
:101AD00003208DF80200C020ADF800006946FE48E2
:101AE000FEF702FD01224021FB48FEF7AEFD012278
:101AF0008021F948FEF7A9FD08BD10B5012280211B
:101B0000F548FEF7A2FD01224021F348FEF79DFDB6
:101B100000228021F048FEF798FD00224021EE4887
:101B2000FEF793FD10BD10B500228021EA48FEF7B4
:101B30008CFD01224021E848FEF787FD012280212B
:101B4000E548FEF782FD10BD70B50546002413E0A0
:101B50008020204100EA05028021DF48FEF775FD64
:101B600001224021DC48FEF770FD00224021DA48C6
:101B7000FEF76BFD601CC4B2082CE9DB012240219A
:101B8000D548FEF762FD00224021D348FEF75DFDF7
:101B900070BD10B50446FFF7B0FF7820FFF7D4FF03
:101BA0000020FFF7D1FF2046FFF7CEFFFFF7BBFF76
:101BB00010BD10B50446FFF7A0FF7820FFF7C4FF63
:101BC0004020FFF7C1FF2046FFF7BEFFFFF7ABFF46
:101BD00010BD70B505460C4645F0B000FFF7D9FFC3
:101BE000102141EA1410FFF7D4FF04F00F00FFF7B3
:101BF000D0FF70BD70B500240EE000212046FFF735
:101C0000E8FF002504E00020FFF7D3FF681CC5B201
:101C1000802DF8DB601CC4B2082CEEDB70BD70B503
:101C20000546691E4906080E0021FFF7D2FF002471
:101C300004E00020FFF7BDFF601CC4B2802CF8DB7D
:101C4000691E012202EB4101C8B20021FFF7C1FF6A
:101C5000002404E00020FFF7ACFF601CC4B2802C1D
:101C6000F8DB70BD2DE9F0410546681EC006070E81
:101C700000240EE039462046FFF7ABFF002604E0C3
:101C80000020FFF796FF701CC6B2082EF8DB601C20
:101C9000C4B2082CEEDBBDE8F0812DE9F041054629
:101CA0000E461746721ED206110E6A1E5206100EFE
:101CB000FFF78FFF002409E0A7F12001874A02EB1C
:101CC0000111085DFFF775FF601CC4B2082CF3DB3F
:101CD000721ED206110E6A1E012303EB4202D0B21D
:101CE000FFF777FF00240BE0A7F120017B4A02EB0E
:101CF000011204F10801505CFFF75BFF601CC4B2E5
:101D0000082CF1DBBDE8F0812DE9F04107460E46D5
:101D10001546002407E02A5D3019C1B23846FFF7A6
:101D2000BCFF601CC4B2285D0028F4D1BDE8F0817E
:101D30002DE9F04105460E461746721E1207110E98
:101D40006A1E5206100EFFF744FF002407E06449A4
:101D500001EB4711085DFFF72CFF601CC4B2102C8B
:101D6000F5DB721E1207110E6A1E012303EB4202FD
:101D7000D0B2FFF72EFF002409E0594901EB4712CA
:101D800004F11001505CFFF714FF601CC4B2102C6A
:101D9000F3DBBDE8F08110B50246012000E05043BE
:101DA0000B1EA1F10101FAD110BD2DE9F0478046CB
:101DB0000E4617461D46002415E0281B411E0A202A
:101DC000FFF7E9FFB7FBF0F00A21B0FBF1F201FBEE
:101DD000120000F130093019C1B24A464046FFF7FF
:101DE0005CFF601CC4B2AC42E7DBBDE8F0872DE9C4
:101DF000F0478146884615461E46002D06DB2B22FD
:101E000041464846FFF749FF2F4605E02D2241464F
:101E10004846FFF742FF6F42002417E0301B411E87
:101E20000A20FFF7B8FFB7FBF0F00A21B0FBF1F290
:101E300001FB120000F1300A08EB0400401CC1B2A3
:101E400052464846FFF729FF601CC4B2B442E5DBA6
:101E5000BDE8F0872DE9F04781460E4690461F46C3
:101E600000241DE0381B411E1020FFF794FFB8FB33
:101E7000F0F000F00F050A2D08DA05F13000C2B2CB
:101E80003019C1B24846FFF708FF07E005F13700F7
:101E9000C2B23019C1B24846FFF7FFFE601CC4B29F
:101EA000BC42DFDBBDE8F0872DE9F04780460E46F7
:101EB00017461D46002419E0281B411E0220FFF78B
:101EC0006AFFB7FBF0F000F0010000F130093019B3
:101ED000C1B24A46404605E0000C0140F845000802
:101EE000E84B0008FFF7D9FE601CC4B2AC42E3DB4C
:101EF000BDE8F08770B5002406E0002500E06D1C09
:101F0000B5F57A7FFBD3641CB4F57A7FF5D3FFF780
:101F1000D7FDAE20FFF73DFED520FFF73AFE80202B
:101F2000FFF737FEA820FFF734FE3F20FFF731FE12
:101F3000D320FFF72EFE0020FFF72BFE4020FFF7F7
:101F400028FEA120FFF725FEC820FFF722FEDA2099
:101F5000FFF71FFE1220FFF71CFE8120FFF719FE7E
:101F6000CF20FFF716FED920FFF713FEF120FFF771
:101F700010FEDB20FFF70DFE3020FFF70AFEA42045
:101F8000FFF707FEA620FFF704FE8D20FFF701FEF6
:101F90001420FFF7FEFDAF20FFF7FBFDFFF72AFE41
:101FA00070BD000008B501210420FEF779FD48202E
:101FB0008DF803000120ADF8000069460B48FEF7DC
:101FC00093FA08BD70B504460D4629462046FEF733
:101FD0001EFB012808D100BF29462046FEF717FB4B
:101FE0000128F9D0012070BD0020FCE70008014065
:101FF00008B501211020FEF753FD8020ADF8000048
:1020000010208DF8030003208DF802006946514826
:10201000FEF76AFA08BD10B5FFF7EAFF80214D48C8
:10202000FEF70FFB10BD08B58020ADF8000048207A
:102030008DF8030069464748FEF756FA08BD08B513
:102040008020ADF8000010208DF8030003208DF8EB
:10205000020069463F48FEF747FA08BD70B5002503
:10206000002424E000BF80213A48FEF7D0FA00287F
:10207000F9D02820FFF788FC80213648FEF7C7FA00
:1020800001280DD100BF80213248FEF7C0FA012897
:10209000F9D0C4F1070101208840C0B2054304E033
:1020A000C4F10701012088408543601CC4B2082C9C
:1020B000D8DB284670BD10B50446FFF7C0FF80216D
:1020C0002448FEF7C0FA44F25060FFF75DFC80211F
:1020D0002048FEF7B6FA1E20FFF756FCFFF7A3FFD5
:1020E00080211C48FEF793FA80BB00BF802119486D
:1020F000FEF78DFA0028F9D000BF80211548FEF7C1
:1021000086FA0128F9D0FFF7A9FF2070FFF7A6FF94
:102110006070FFF7A3FFA070FFF7A0FFE070FFF76C
:102120009DFF2071FFF78BFF80210A48FEF789FA97
:10213000207861780844A1780844E178084421793E
:10214000884201D1012010BD0020FCE7FFE70020FC
:10215000F9E700000010014008B501210420FEF756
:102160009FFC1020ADF8000003208DF80200102025
:102170008DF8030069460748FEF7B6F910210548B7
:10218000FEF761FA08BD10B510210248FEF74CFABF
:1021900010BD00000008014008B54FF4A060FEF734
:1021A000D5F825208DF8000001208DF801008DF86C
:1021B00002008DF803006846FEF7CDF808BD00B5B3
:1021C00085B001210420FEF76BFC01218803FEF796
:1021D00067FC4FF40070ADF8100018208DF8130064
:1021E00003208DF8120004A95548FEF77DF94FF43D
:1021F0008060ADF8100004208DF8130004A9504849
:10220000FEF772F94FF4E13000900020ADF80400C1
:10221000ADF80600ADF80800ADF80C000C20ADF8E4
:102220000A0069464748FEF7E2FCFFF7B5FF0122C6
:1022300040F225514348FEF772FD012240F224414D
:102240004048FEF76CFD01213E48FEF75CFD05B0FD
:1022500000BD70B504460D4629462046FEF7C0FD78
:1022600000BF80212046FEF729FE0028F9D070BD6E
:102270002DE9F04107460D461646002405E0295D8C
:102280003846FFF7E6FF601CC4B2B442F7DB00BF7C
:1022900040213846FEF712FE0028F9D0BDE8F08153
:1022A00070B506460C46002500BF615D3046FFF75D
:1022B000D0FF6D1C605D0028F7D100BF4021304683
:1022C000FEF7FCFD0028F9D070BD2DE9F041054670
:1022D0000C46260AE7B231462846FEF781FD00BFCC
:1022E00080212846FEF7EAFD0028F9D03946284625
:1022F000FEF776FD00BF80212846FEF7DFFD0028AF
:10230000F9D0BDE8F08170B504460D46E1B20D4844
:10231000FEF766FD00BF80210A48FEF7CFFD0028CA
:10232000F9D0204670BD10B5044600BF20210548F5
:10233000FEF7C4FD0028F9D00248FEF755FD10BD98
:10234000000801400038014010B504462246012132
:102350005948FEF77AF910BD10B5044622462021EF
:102360005648FEF772F910BD10B50446224680218A
:102370005248FEF76AF910BD10B540214F48FEF7EC
:1023800046F910BD08B501210420FEF789FB0121A3
:102390001020FEF785FB10208DF80300A020ADF87B
:1023A000000003208DF8020069464448FEF79CF8BF
:1023B00010208DF803000120ADF8000003208DF8F7
:1023C000020069463C48FEF78FF848208DF803006C
:1023D0004020ADF8000003208DF802006946374820
:1023E000FEF782F80120FFF7AFFF0020FFF7B4FFF0
:1023F00008BD10B50020FFF7A7FF10BD10B50120E4
:10240000FFF7A2FF10BDF8B505460026002432E014
:1024100080212141294009B1012100E00021084625
:10242000FFF7A2FF0020009002E00098401C0090FF
:1024300000980A28F9DB0120FFF78EFF00200090AA
:1024400002E00098401C009000980A28F9DBFFF792
:1024500093FF10B18020204106430020FFF77CFF4E
:102460000020009002E00098401C009000980A288C
:10247000F9DB601CC4B2082CCADB3046F8BD70B56D
:102480000446002513E004F08000FFF76DFF6006AE
:10249000040E0120FFF760FFFFF76EFF012801D156
:1024A00044F001040020FFF757FF681CC5B2082D57
:1024B000E9DB204670BD000000100140000801402B
:1024C00010B5FFF75FFF10BD70B505460C46FFF76E
:1024D00090FF9F20FFF797FFFF20FFF794FF2870E2
:1024E000FF20FFF790FF208020884FF6FF7101EA60
:1024F00000202080FF20FFF786FF218808432080EE
:10250000FFF77CFF70BD10B5FFF773FF0620FFF7E4
:102510007AFFFFF773FF10BD70B50024FFF769FF66
:102520000520FFF770FF3F4D10E06D1E641CB4F5F1
:102530007A7F09D3FFF762FFFEF72DF9FFF759FF06
:102540000520FFF760FF002405B906E0FF20FFF734
:102550005AFF00F001000028E7D100BFFFF74EFF4F
:1025600070BD2DE9F04104460E461746FFF7CBFF3C
:10257000FFF73FFF0220FFF746FFC4F30740FFF7D6
:1025800042FFC4F30720FFF73EFFE0B2FFF73BFF37
:10259000002504E0705DFFF736FF681C85B2BD4280
:1025A000F8DBFFF72BFFFFF7B7FFBDE8F08110B5B1
:1025B0000446FFF7A8FFFFF71CFF2020FFF723FFCB
:1025C000C4F30740FFF71FFFC4F30720FFF71BFF0B
:1025D000E0B2FFF718FFFFF711FFFFF79DFF10BDF7
:1025E0002DE9F04104460E461746FFF702FF03208F
:1025F000FFF709FFC4F30740FFF705FFC4F3072007
:10260000FFF701FFE0B2FFF7FEFE002504E0FF2028
:10261000FFF7F9FE70556D1CBD42F8D3FFF7EEFED3
:10262000BDE8F081A086010010B500F0D1F90446A4
:1026300024B1012C04D0052C06D103E0002010BDEC
:102640000120FCE70120FAE70120F8E700207047AD
:1026500070B504460D462946204600F051FA06465C
:1026600036B1012E06D0022E06D0042E08D105E088
:10267000002070BD0120FCE70220FAE70420F8E703
:102680000120F6E73EB504460CB904203EBD68467D
:1026900000F0B8FA0546DDB9009820609DF8040006
:1026A00020719DF8050060719DF80600A0719DF8ED
:1026B0000700E0719DF8080020729DF80900607223
:1026C0009DF80A00A0729DF80B10E1720020DDE772
:1026D000012D04D0032D04D0042D06D103E00120E8
:1026E000D4E70320D2E70420D0E70120CEE710B5DD
:1026F00000F0CCFA044614B1012C04D101E0002012
:1027000010BD0120FCE70120FAE710B500F0DDFA6A
:1027100010BD10B500F0D6FA10BD10B500F0CFFA1C
:1027200010BD3EB555A001F003FDFFF7EEFF0028F8
:102730003FD06846FFF7A6FF0446002C34D15BA0CB
:10274000009901F0F5FC9DF807209DF806105CA0AB
:1027500001F0EEFC9DF805209DF804105DA001F04D
:10276000E7FC9DF8081060A001F0E2FC9DF809006C
:10277000AA2801D161A000E062A0014663A001F097
:10278000D7FCFFF7C6FF0546294665A001F0D0FC3F
:10279000FFF7C3FF08B967A000E06AA00546294615
:1027A0006DA001F0C5FC07E0214670A001F0C0FC5F
:1027B00002E078A001F0BCFC7CA001F0B9FC3EBDB9
:1027C000FEB506460C460CB90420FEBD69463046EF
:1027D00000F032FA0546DDB9009820609DF804004B
:1027E00020719DF8050060719DF80600A0719DF8AC
:1027F0000700E0719DF8080020729DF809006072E2
:102800009DF80A00A0729DF80B10E1720020DCE731
:10281000012D04D0032D04D0042D06D103E00120A6
:10282000D3E70320D1E70420CFE70120CDE770B53F
:102830000446204600F02EFA054615B1012D04D1BC
:1028400001E0002070BD0120FCE70120FAE710B58F
:1028500000F000FC10BD10B500F03EFA10BD10B540
:1028600000F012F9044614B1012C04D101E000205B
:1028700010BD0120FCE70120FAE700000D0A3D3DF4
:102880003D20573235513634E4B8ADE5AD98E58298
:10289000A8E79A84E69C80E696B04448543131E635
:1028A00095B0E68DAE203D3D3D0D0A00E697B6E9B8
:1028B00097B4E688B33A202564E7A7925C720A00D1
:1028C000E6B8A9E5BAA63A2025642E2564E28483F9
:1028D0005C720A00E6B9BFE5BAA63A2025642E2547
:1028E00064252552480D0A00E6A0A1E9AA8CE592CC
:1028F0008C3A203078253032580D0A00E69C89E663
:1029000095880000E697A0E695880000E695B0E679
:102910008DAEE78AB6E680813A2025730D0A000065
:10292000E680BBE8AEB0E5BD95E695B03A202564FB
:102930000D0A0000E8A686E79B96E6A8A1E5BC8FF5
:1029400000000000E78EAFE5BDA2E7BC93E586B2CC
:10295000E6A8A1E5BC8F0000E5AD98E582A8E6A851
:10296000A1E5BC8F3A2025730D0A0000E8AFBBE556
:102970008F96E695B0E68DAEE5A4B1E8B4A5EFBCC0
:102980008CE99499E8AFAFE7A0813A2025640D0A5D
:1029900000000000E69A82E697A0E69C89E695880A
:1029A000E695B0E68DAE0D0A000000003D3D3D3DD0
:1029B0003D3D3D3D3D3D3D3D3D3D3D3D3D3D3D3D47
:1029C0003D3D3D3D3D3D3D3D3D3D3D3D0D0A000014
:1029D0001CB5FFF775FD694601A8FFF775FD9DF869
:1029E0000400EF2805D1BDF8000044F21701884229
:1029F00008D0BDF800209DF80410D6A001F098FB87
:102A000005201CBDBDF800209DF80410DEA001F0DB
:102A10008FFB2822E9494FF48030FFF7E1FDE748BA
:102A20000068E74988421ED0E6A001F081FB28211A
:102A3000E24801F0F6FAE248E04908600020486008
:102A40008860C8600861486108764FF48030FFF7FD
:102A5000AEFD2822D9494FF48030FFF782FDE8A06F
:102A600001F066FB04E0D5484168EDA001F060FB91
:102A70000120F84908700020C3E7F648007808B93B
:102A8000012070470020FCE770B5F3A001F050FB77
:102A9000002409E025032846FFF789FD1022611C68
:102AA000F7A001F045FB641C102CF3DB2821C34880
:102AB00001F0B7FAC248C149086000204860886048
:102AC000C8600861486108764FF48030FFF76FFDF9
:102AD0002822BA494FF48030FFF743FDEEA001F001
:102AE00027FB002070BD10B54FF48030FFF75FFD6D
:102AF0002822B2494FF48030FFF733FD002010BD8B
:102B0000FEB504460F46D348007808B90120FEBD43
:102B10000CB90420FBE7009720788DF8040060785A
:102B20008DF80500A0788DF80600E0788DF8070094
:102B300020798DF80800AA208DF8090000208DF872
:102B40000A0000218DF80B109C48007E90B90025EA
:102B50009A48406810B10020FFF729FD0C22694611
:102B60002846FFF7FEFC012094494860084645616D
:102B7000056143E09148C168806801EB00358F48EA
:102B8000C0680C30B0F5805F14D98C488068401C58
:102B90008A4988600020C86008468068102801D3F0
:102BA000002088608548806806033046FFF7FFFCF8
:102BB000354600BF0C2269462846FFF7D2FC7F4805
:102BC0004561C0680C307D49C8600846406841F2E4
:102BD0005051884205D279484068401C7749486086
:102BE0000CE005F10C0075490861084600694FF6D4
:102BF000FF71884202D3002070490861FFF773FF1C
:102C0000002084E710B504469248007800B10CB962
:102C1000042010BD6948406808B90320F9E76749F6
:102C20000C2248692146FFF7DBFC607AAA2801D014
:102C30000120EEE70020ECE770B504460E4685481B
:102C4000007800B10EB9042070BD5C484068A04215
:102C500001D80420F8E75948007E20B90CB10420BF
:102C6000F2E7002506E05548406904EB4401A0EB7B
:102C7000810500BF0C2231462846FFF7B1FC707A6F
:102C8000AA2801D00120DFE70020DDE710B5FFF71B
:102C9000FBFE10BD10B504466E48007808B901204F
:102CA00010BD46480476FFF71EFF0CB984A000E073
:102CB00087A001468BA001F03BFA0020F0E73F48D7
:102CC000007E70473D48406870473C48406808B106
:102CD000012070470020FCE710B58AA001F028FA17
:102CE0003648016891A001F023FA3448416895A064
:102CF00001F01EFA3148007E08B971A000E074A00E
:102D0000014695A001F014FA2C48816897A001F0C3
:102D10000FFA2A48C1689AA001F00AFA27484169C7
:102D20009EA001F005FA25480169A4A001F000FA6F
:102D300041F25051A9A001F0FBF90C21AFA001F024
:102D4000F7F94021B5A001F0F3F9BBA001F0F0F9CB
:102D500010BD0000573235513634E88AAFE7898715
:102D6000E6A380E6B58BE5A4B1E8B4A521204D49E2
:102D7000443D3078253032582C204449443D307849
:102D8000253034580D0A0000573235513634E88A60
:102D9000AFE78987E6A380E6B58BE68890E58A9F52
:102DA00021204D49443D3078253032582C2044496B
:102DB000443D3078253034580D0A0000780000205A
:102DC00078563412E6A380E6B58BE588B0E9A6967E
:102DD000E6ACA1E4BDBFE794A8EFBC8CE6ADA3E5EB
:102DE0009CA8E5889DE5A78BE58C96E5AD98E582E6
:102DF000A8E58CBAE59F9F2E2E2E0D0A000000003C
:102E0000E5AD98E582A8E58CBAE59F9FE5889DE54C
:102E1000A78BE58C96E5AE8CE688905C720A000084
:102E2000E8AFBBE58F96E588B0E5AD98E582A8E709
:102E3000AEA1E79086E4BFA1E681AFEFBC8CE6804F
:102E4000BBE8AEB0E5BD95E695B03A2025640D0A25
:102E5000000000003E000020E5BC80E5A78BE6A056
:102E6000BCE5BC8FE58C96573235513634E5AD98CC
:102E7000E582A8E58CBAE59F9F2E2E2E0D0A000054
:102E8000E5B7B2E693A6E999A4E68987E58CBA206E
:102E900025642F25640D0A00573235513634E5ADCF
:102EA00098E582A8E58CBAE59F9FE6A0BCE5BC8FBB
:102EB000E58C96E5AE8CE68890210D0A00000000B6
:102EC000E8A686E79B96E6A8A1E5BC8F0000000077
:102ED000E78EAFE5BDA2E7BC93E586B2E6A8A1E523
:102EE000BC8F0000E5AD98E582A8E6A8A1E5BC8FFF
:102EF000E5B7B2E8AEBEE7BDAEE4B8BA3A20257396
:102F00000D0A00000D0A3D3D3D2057323551363443
:102F1000E5AD98E582A8E7B3BBE7BB9FE4BFA1E6B8
:102F200081AF203D3D3D0D0A00000000E9AD94E673
:102F300095B0E6A087E8AF863A203078253038583B
:102F40000D0A0000E680BBE8AEB0E5BD95E695B0A1
:102F50003A2025640D0A0000E5AD98E582A8E6A8B0
:102F6000A1E5BC8F3A2025730D0A0000E5BD93E56D
:102F7000898DE68987E58CBA3A2025640D0A000020
:102F8000E5BD93E5898DE5818FE7A7BB3A202564F0
:102F9000E5AD97E88A820D0A00000000E69C80E615
:102FA00096B0E8AEB0E5BD95E59CB0E59D803A20D1
:102FB0003078253038580D0A00000000E69C80E685
:102FC00097A7E8AEB0E5BD95E59CB0E59D803A20B9
:102FD0003078253038580D0A00000000E69C80E566
:102FE000A4A7E8AEB0E5BD95E5AEB9E9878F3A2074
:102FF0002564E69DA15C720A00000000E58D95E65F
:103000009DA1E8AEB0E5BD95E5A4A7E5B08F3A2057
:103010002564E5AD97E88A820D0A0000E58886E917
:10302000858DE5AD98E582A8E7A9BAE997B43A207D
:1030300025644B420D0A00003D3D3D3D3D3D3D3D7B
:103040003D3D3D3D3D3D3D3D3D3D3D3D3D3D3D3DB0
:103050000D0A000030B587B01FA001F069F82948BB
:103060004168AFF2201001F063F82648406838B993
:1030700025A001F05DF82AA001F05AF807B030BD94
:1030800000251FE004A92846FFF7D6FD04469CB999
:103090009DF818009DF815109DF814209DF8173024
:1030A000CDE90032CDE902109DF8163029462448BA
:1030B000049A01F03DF804E02246294621A001F0DF
:1030C00037F86D1C0F484068A842DBD814A001F007
:1030D0002FF800BFD2E700000D0A3D3D3D205732DA
:1030E00035513634E4B8ADE79A84E68980E69C89A8
:1030F0004448543131E695B0E68DAE203D3D3D0D5E
:103100000A00000078000020E69A82E697A0E69583
:10311000B0E68DAEE8AEB0E5BD950D0A000000004A
:103120003D3D3D3D3D3D3D3D3D3D3D3D3D3D3D3DCF
:103130003D3D3D3D3D3D3D3D3D3D3D3D3D0D0A005F
:10314000484F0008E8AEB0E5BD952025643A20E878
:10315000AFBBE58F96E5A4B1E8B4A52028E9949922
:10316000E8AFAFE7A0813A202564290D0A000000EE
:1031700008B54FF4A060FDF7E9F827208DF80000AE
:1031800000208DF801008DF8020001208DF8030069
:103190006846FDF7E0F808BD00B585B00121880458
:1031A000FDF78BFC01210820FDF77AFC4FF48060CD
:1031B000ADF8100018208DF8130003208DF81200D0
:1031C00004A9F948FDF790F94FF40060ADF810003C
:1031D00004208DF8130004A9F348FDF785F94FF496
:1031E000E13000900020ADF80400ADF80600ADF825
:1031F0000800ADF80C000C20ADF80A006946EB4859
:10320000FDF7F5FC012240F22551E848FDF787FD66
:10321000012240F22441E548FDF781FDFFF7A8FFB8
:103220000121E248FDF76FFD05B000BD08B50121A1
:103230000820FDF735FC4FF48070ADF80000102039
:103240008DF8030003208DF802006946D648FDF78B
:103250004BF901210820FDF723FC4FF40070ADF875
:1032600000006946D048FDF73FF908BD10B5FFF7EB
:10327000DDFFFFF791FF4FF40071CB48FDF7E1F957
:103280004FF48071C848FDF7DEF910BD10B54FF45A
:103290000071C548FDF7D7F9C548FEF775FB4FF437
:1032A0000071C148FDF7CDF910BD2DE9F04106468A
:1032B0000C4615461F46BF48B0F800046FF30E00D9
:1032C000BC49A1F800043246BBA1B848FEF7C7FAD2
:1032D0001CB915B90120BDE8F0814FF47A7107FBE4
:1032E00001F0FEF751FB0020B249B1F80014C1F320
:1032F0000E01B04A50541146B1A000F019FFAD487C
:10330000B0F800046FF30E00AA49A1F800040846C3
:10331000B0F8000420F40040A1F80004B4B1ADB14D
:103320002146A44800F088FE08B1012000E00020FA
:1033300040B929469F4800F07FFE08B1012000E017
:10334000002008B10120C6E70020C4E744B12146AF
:10335000984800F071FE08B10120BCE70020BAE7F0
:103360002946944800F068FE08B10120B3E7002028
:10337000B1E710B500244FF400718B48FDF761F9F7
:1033800090A000F0D5FE9448FEF7FEFA15E0214625
:1033900092A000F0CDFE4FF4FA73002296A197A000
:1033A000FFF783FF28B1214695A000F0C1FE012060
:1033B00010BDFFF76BFF601CC4B20A2CE7DB0020D6
:1033C000F6E710B5044624B1012C0AD0022C18D11E
:1033D0000FE040F6C41393A287A195A0FFF765FF05
:1033E00010BD40F6C4138FA283A194A0FFF75DFF28
:1033F000F6E740F6C4138BA27FA193A0FFF755FF19
:10340000EEE70020ECE700B58BB092A101A800F038
:103410009FFE4FF4FA73002277A101A8FFF745FF42
:103420000BB000BD30B59FB004460D462B4622467A
:103430008DA101A800F08CFE41F2883300226EA11C
:1034400001A8FFF732FF1FB030BD70B5A0B0044631
:103450000D4616462B46224688A102A8009600F08B
:1034600077FE4FF47A73002263A102A8FFF71DFFD5
:1034700020B070BD10B586B004460CB1012000E04C
:103480000020024683A101A800F062FE4FF4FA7307
:10349000002259A101A8FFF708FF06B010BDF0B542
:1034A000B9B006460F4614461D46642120A800F018
:1034B000B8FD16B1012E10D107E03B4679A27AA1E2
:1034C00020A8009400F044FE08E03B467AA276A1D2
:1034D00020A8009400F03CFE00E000BF00BF052DD6
:1034E00006DA20AB2A4675A102A800F031FE04E0FE
:1034F00020AA77A102A800F02BFE4FF47A6378A2ED
:103500003DA102A8FFF7D1FE39B0F0BD70B5BCB047
:1035100004460D461646FCB12B46012274A11EA896
:1035200000F016FE324677A1684600F011FE4FF417
:10353000FA73002230A11EA8FFF7B7FE50B14FF476
:10354000FA7300222CA16846FFF7AFFE10B10120EC
:103550003CB070BD0020FBE72B46002264A11EA8F2
:1035600000F0F6FD4FF4FA73002223A11EA8FFF726
:103570009CFEEDE710B54FF4FA7300221EA165A082
:10358000FFF793FE68B167A10A4800F055FD08B146
:10359000022010BD66A1074800F04EFD10B10320C7
:1035A000F7E7D2E0CAE00000000C0140004800400C
:1035B00020A10700A000002025730D0A00000000D4
:1035C000257300000D0A4154E6B58BE8AF952E2E09
:1035D0002E2E2E0D0A00000080841E000D0A41547C
:1035E000E6B58BE8AF95E6ACA1E695B02025642E54
:1035F0002E2E2E2E2E0D0A004F4B0000415400009F
:103600000D0A4154E6B58BE8AF95E590AFE58AA881
:10361000E68890E58A9F2025642E2E2E2E2E2E0DD4
:103620000A0000006E6F206368616E67650000002D
:1036300041542B43574D4F44453D310041542B439A
:10364000574D4F44453D320041542B43574D4F4455
:10365000453D330041542B4357444843505F435545
:10366000523D312C3100000041542B43574A415008
:103670003D222573222C22257322000041542B4326
:10368000575341503D222573222C222573222C3181
:103690002C25640041542B4349504D55583D256419
:1036A0000000000054435000222573222C22257371
:1036B000222C2573000000005544500041542B4338
:1036C000495053544152543D25642C257300000049
:1036D00041542B43495053544152543D25730000EB
:1036E000414C5245415920434F4E4E4543540000F2
:1036F00041542B4349505345525645523D25642C65
:103700002573000041542B43495053544F3D2573BA
:103710000000000041542B43495053544154555329
:10372000000000005354415455533A320D0A000032
:103730005354415455533A330D0A00007BA17E483F
:1037400000F07AFC08B1042023E7002021E710B53F
:1037500000244FF4FA730022AFF26411AFF24C0070
:10376000FFF7A3FD002831D074A1734800F064FC7A
:1037700010B144F0010401E024F0010473A16E488B
:1037800000F05AFC10B144F0020401E024F00204FD
:1037900072A1694800F050FC10B144F0040401E04B
:1037A00024F0040471A1644800F046FC10B144F018
:1037B000080401E024F0080470A15F4800F03CFC1C
:1037C00010B144F0100401E024F01004204610BDB4
:1037D0002DE9F04105460F464FF4FA730022AFF28F
:1037E000E8116AA0FFF761FD6BA1534800F024FCCB
:1037F00006460EB1B61D02E00020BDE8F0810024AF
:1038000009E0305D2855285D222802D10020285586
:1038100003E0601CC4B2BC42F3DB00BF0120ECE754
:1038200010B54FF4FA730022AFF234215CA0FFF719
:103830003CFD08B9002010BD4FF4FA735CA2AFF252
:1038400048215CA0FFF731FDF5E710B55C48FEF7B5
:103850009BF85CA15C48FEF702F85C48FEF794F820
:1038600010BD2DE9F04186B007460C4615461E46B0
:103870004FF0000847B12246AFF2BC215248FDF795
:10388000EEFF4FF001081CE0052E06DAAB1C3246B5
:103890004FA101A800F05CFC04E0AA1C51A101A802
:1038A00000F056FC4FF47A73002252A101A8FFF7F2
:1038B000FCFC4FF47A7300224FA12046FFF7F5FC81
:1038C000804641464EA000F033FC404606B0BDE8BD
:1038D000F08170B5044600251748B0F800046FF376
:1038E0000E001549A1F800040846B0F8000420F4C1
:1038F0000040A1F8000400BF0F48B0F80004C00B5E
:103900000028F9D000200C49B1F80014C1F30E01D1
:10391000094A50540CB1154605E03DA1064800F097
:103920008BFB00B1044D284670BD00005354415438
:1039300055533A340D0A0000A00000202B43495093
:103940005354415455533A302C0000002B434950F6
:103950005354415455533A312C0000002B434950E5
:103960005354415455533A322C0000002B434950D4
:103970005354415455533A332C0000002B434950C3
:103980005354415455533A342C00000041542B43B6
:103990004946535200000000415049502C2200007B
:1039A00041542B4349504D4F44453D3100000000E8
:1039B0003E00000041542B43495053454E44000003
:1039C00040420F002B2B2B000048004020A1070095
:1039D00041542B43495053454E443D25642C2564A6
:1039E0000000000041542B43495053454E443D25AF
:1039F000640000003E20000053454E44204F4B0021
:103A0000E8BF94E59B9EE580BCEFBC9A256400006E
:103A10002B49504400000000F0B589B00546202134
:103A200001A800F0FEFA00270026284600F016FB49
:103A3000C7B2642F00DD642700240DE0F34850F87E
:103A40002410284600F0F8FA08B1012000E0002018
:103A500000B103E0601CC4B2082CEFDB00BF002003
:103A60000DE0295C202908DB295C7E2905DC2B5C24
:103A70003146721CD6B201AA5354411CC8B2B84296
:103A800001DA1E2EEDDB002001A98855E0A000F030
:103A90004FFB0420FEF7C3F8082C07DADB4850F888
:103AA000242001210420FEF72FF90CE0002E05DD73
:103AB00001AA01210420FEF727F904E0D8A2012180
:103AC0000420FEF721F9082C51D2DFE804F0040DA0
:103AD00018222B353F472020D34908600120091FB9
:103AE00008600220086043E02020CF49091F0860D9
:103AF0000120091D08600220091F086038E020200D
:103B0000C949091F0860012008600220091D0860DA
:103B10002EE02020C4490860012008600220091F0F
:103B2000086025E02020C04908600120091F0860C6
:103B30000220091D08601BE02020BB49091F086006
:103B40000120091D08600220086011E02020B6490C
:103B50000860012008600220086009E02020B249C6
:103B6000091F0860012008600220086000E000BF13
:103B700000BF09B0F0BD10B5ACA000F0D9FAB3A0F9
:103B800000F0D6FA4FF48071A7481438FCF759FDBD
:103B900001E0FCF700FEFFF7ECFB0028F9D001E0A4
:103BA000FCF7F9FDFFF72FFC0028F9D0AEA000F0DC
:103BB000BFFA01E0FCF7EFFD0020FFF702FC002850
:103BC000F8D0B3A000F0B4FA01E0FCF7E4FDB8A12E
:103BD000BAA0FFF727FC0028F7D0BAA000F0A8FA97
:103BE00001E0FCF7D8FD0020FFF744FC0028F8D0E6
:103BF000BBA000F09DFA01E0FCF7CDFD0523C0A2BB
:103C0000C1A10020FFF74BFC0028F5D0C2A000F0B6
:103C10008FFA01E0FCF7BFFDFFF702FE0028F9D0A4
:103C2000C6A000F085FA10BD10B59CB0642103A8B1
:103C300000F0F7F9C848006801280DD1C748C078DE
:103C4000C6498978CDE90010C44843780278C44950
:103C500003A800F07DFA03E0C2A103A800F078FAFF
:103C600003A9C5A000F064FA0523002203A90120DE
:103C7000FFF7F7FDC148007800282CD0FFF7E5FDDD
:103C800000BFFFF777FC0446FCF785FD002CF8D059
:103C9000042C19D1BAA000F04BFA01E0FCF77BFD2F
:103CA00083A186A0FFF7BEFB0028F7D001E0FCF758
:103CB00072FD052392A294A10020FFF7F0FB0028DB
:103CC000F5D0BAA000F034FA01E0FCF764FDFFF78C
:103CD000A7FD0028F9D01CB010BD70B5BC48B0F8E5
:103CE00000040121B1EBD03F30D10020B849B1F838
:103CF0000014C1F30E01B64A50541046FFF78CFE73
:103D000000240DE0B248015DB248FDF769F800BF3C
:103D10004021B048FDF7D2F80028F9D0601C84B2E9
:103D2000AB48B0F80004C0F30E00A042EADCA8489B
:103D3000B0F800046FF30E00A549A1F8000408468E
:103D4000B0F8000420F40040A1F80004A248B0F844
:103D50000004C00B80B300209F49B1F80014C1F3E8
:103D60000E019D4A50541046FFF756FE00240DE008
:103D70009948015D9948FDF733F800BF4021974805
:103D8000FDF79CF80028F9D0601C84B29248B0F886
:103D90000004C0F30E00A042EADC8F48B0F8000433
:103DA0006FF30E008C49A1F800040846B0F8000437
:103DB00020F40040A1F8000470480078002824D0C6
:103DC000FFF743FD00BFFFF7D5FB0546002DFAD0F6
:103DD000042D15D16AA000F0ABF900BF34A137A0C3
:103DE000FFF720FB0028F9D000BF052344A246A11D
:103DF0000020FFF754FB0028F7D06CA000F098F9E2
:103E000000BFFFF70DFD0028FBD070BD4000002073
:103E100052656365697665643A2025730D0A000072
:103E20004E4F5F434D440000140C01400D0AE6ADB7
:103E3000A3E59CA8E9858DE7BDAE204553503832F7
:103E40003636202E2E2E2E2E2E0D0A000D0AE4BD03
:103E5000BFE883BD2045535038323636202E2E2EF3
:103E60002E2E2E0D0A0000000D0AE6ADA3E59CA83B
:103E7000E9858DE7BDAEE5B7A5E4BD9CE6A8A1E563
:103E8000BC8F20535441202E2E2E2E2E2E0D0A0094
:103E90000D0AE6ADA3E59CA8E8BF9EE68EA52057D7
:103EA000694669202E2E2E2E2E2E0D0A00000000AF
:103EB0003135303336313138313735003231313503
:103EC000000000000D0AE7A681E6ADA2E5A49AE88D
:103ED000BF9EE68EA5202E2E2E2E2E2E0D0A000021
:103EE0000D0AE6ADA3E59CA8E8BF9EE68EA520538B
:103EF0006572766572202E2E2E2E2E2E0D0A000053
:103F000038303030000000003139322E3136382E52
:103F1000312E3131000000000D0AE8BF9BE585A578
:103F2000E9808FE4BCA0E58F91E98081E6A8A1E556
:103F3000BC8F202E2E2E2E2E2E0D0A000D0AE98566
:103F40008DE7BDAE204553503832363620E5AE8C75
:103F5000E6AF950D0A00000034000020600000204C
:103F6000984F00085265616420444854313120451F
:103F700052524F52210D0A002573000065000020A7
:103F80000D0AE6ADA3E59CA8E9878DE8BF9EE7830F
:103F9000ADE782B9E5928CE69C8DE58AA1E599A80A
:103FA000202E2E2E2E2E2E0D0A0000000D0AE9873F
:103FB0008DE8BF9EE783ADE782B9E5928CE69C8DE4
:103FC000E58AA1E599A8E68890E58A9F0D0A000098
:103FD000A204002000480040A0000020003801405A
:103FE00010B50120FCF7E2FC00BF6120FCF72DFCBE
:103FF0000028FAD045F25550FCF7C4FB0620FCF728
:10400000C4FB40F63440FCF7C3FBFCF7C4FBFCF7F1
:10401000C7FB10BDD2B201E000F8012B491EFBD254
:1040200070470022F6E710B513460A4604461946C3
:10403000FFF7F0FF204610BD30B505462A460B4677
:1040400012F8010B13F8014B08B1A042F8D01CB1D3
:10405000002802D06D1CF1E7284630BD421C10F844
:10406000011B0029FBD1801A70472DE9F05F05463E
:10407000002092469B4688460646814640241BE027
:10408000284641464746224600F041F853465A46E4
:10409000C01A914110D311461846224600F028F864
:1040A0002D1A67EB01084F4622460120002100F03F
:1040B0001FF817EB00094E41201EA4F10104DFDCBC
:1040C000484631462A464346BDE8F09F064C074D18
:1040D00006E0E06840F0010394E8070098471034D8
:1040E000AC42F6D3FCF728F83C5000085C500008BE
:1040F000202A04DB203A00FA02F1002070479140A8
:10410000C2F1200320FA03F3194390407047202A9C
:1041100004DB203A21FA02F00021704721FA02F371
:10412000D040C2F120029140084319467047000078
:104130000FB4054B10B503A9044A029800F02CF8FF
:1041400010BC5DF814FB0000072300086800002085
:104150000FB4084B10B504A902AA039800F01CF88C
:10416000044602A9002000F042FA204610BC5DF887
:1041700014FB0000EF45000802E008C8121F08C148
:10418000002AFAD170477047002001E001C1121FD8
:10419000002AFBD1704700002DE9FF4F8DB00F467C
:1041A0000546002606E025280BD0DDE90F129047D2
:1041B0006D1C761C28780028F5D111B03046BDE87A
:1041C000F08F0024A246A1460122E94900E0044301
:1041D00015F8013F203B02FA03F00842F7D1287896
:1041E0002A2810D06FF02F022878A0F13001092979
:1041F00014D80AEB8A0102EB410144F0020400EBFF
:10420000010A6D1CF0E701CF5FEA000A03D544F410
:104210000054CAF1000A44F002046D1C28782E28CC
:1042200017D115F8010F44F004042A280ED06FF0BE
:104230002F022878A0F1300109290AD809EB890159
:1042400002EB410100EB01096D1CF2E757F8049BFA
:104250006D1C28786C280FD006DC4C2817D06828F5
:104260000DD06A2814D104E0742810D07A280FD118
:104270000DE044F400140AE044F4801401E044F436
:1042800040146978814202D104F580146D1C6D1CC4
:1042900028786E281ED00CDC632830D004DC00287F
:1042A0008BD0582811D19FE0642867D069280CD1A1
:1042B00064E073282DD004DC6F2872D0702804D1FC
:1042C00094E075286ED078286DD0DDE90F12904704
:1042D000761C4BE1C4F30250022806D0032809D013
:1042E000042801CF09D0066040E101CFF117C0E9F1
:1042F00000613BE101CF068038E1067036E117F836
:10430000040B8DF8000000208DF80100EB46012021
:1043100003E057F804BB4FF0FF3061074FF0000196
:1043200002D40DE008F10101884649450FDA8045C5
:10433000F8DB1BF808100029F4D108E008F10101AE
:1043400088468142FADB1BF808100029F6D1DDE926
:104350000F23AAEB08008146214600F031F93044D2
:1043600000EB080604E0DDE90F121BF8010B904793
:10437000B8F10108F7D221464846F2E00A21C4F319
:1043800002524FF0000B0891022A04D001CFC1174E
:10439000032A09D00AE0FF1D27F00707F7E802010A
:1043A00008E02CE01EE01FE000B2C117042A01D192
:1043B00040B2C117021E71F1000206DA0023D0EBF1
:1043C000030063EB01012D2202E0220504D52B221C
:1043D0008DF82420012203E0E20701D02022F7E734
:1043E000904653E00A210BE0102109E010214FF024
:1043F000000B44F004044FF00809089103E0082181
:104400004FF0000B0891C4F30252022A04D001CFEE
:104410000021032A06D006E0FF1D27F00707F7E872
:10442000020103E080B2042A00D1C0B24FF00008BC
:1044300022072BD52A78702A07D0DDF820C08CF00F
:10444000100C5CEA0B0C05D00EE040228DF8242005
:10445000012208E050EA010306D030238DF8243011
:104460008DF8252002229046089B83F0080353EA2A
:104470000B030BD150EA010201D1620706D53022AD
:104480008DF824204FF00108A9F101092A78582A53
:1044900004D038A20B9208AA0A920BE03AA2F9E7DC
:1044A0005B46089AFFF7E1FD0B9B9B5C0A9A521E44
:1044B0000A92137050EA0102F2D10A98ADEB0000A3
:1044C00000F1200B600702D524F4803401E04FF0A6
:1044D0000109D94502DDA9EB0B0000E0002000EB4B
:1044E0000B0141440890AAEB010AE00306D4DDE980
:1044F0000F232146504600F063F806444FF00009B0
:1045000008E009A911F80900DDE90F12904709F147
:104510000109761CC145F4DBE0030CD5DDE90F236E
:104520002146504600F04CF8064404E0DDE90F1245
:1045300030209047761C0899481E08900029F5DC29
:1045400008E00A980A990078491C0A91DDE90F12DF
:104550009047761CBBF10001ABF1010BF1DC214669
:104560005046DDE90F2300F019F806446D1C21E6E2
:104570000928010030313233343536373839616239
:1045800063646566000000003031323334353637FD
:104590003839414243444546000000002DE9F041CE
:1045A000044600251E461746880404D405E0394613
:1045B0002020B0476D1C641EF9D52846BDE8F08167
:1045C0002DE9F041044600251E469046C80301D55A
:1045D000302700E02027880404D505E0414638460E
:1045E000B0476D1C641EF9D52846BDE8F0810A6805
:1045F000531C0B60107070470000000000000000AA
:104600000000000000000000000000F800000000B2
:10461000000000333000000000100C06100C0600F3
:10462000000000000000000040C07840C07840005A
:10463000043F04043F040400007088FC08300000BC
:10464000001820FF211E0000F008F000E018000014
:1046500000211C031E211E0000F0088870000000CD
:104660001E2123241927211010160E00000000001F
:104670000000000000000000000000E0180402003C
:10468000000000071820400000020418E0000000AD
:104690000040201807000000404080F080404000AB
:1046A0000202010F01020200000000F00000000001
:1046B0000101011F010101000000000000000000D5
:1046C00080B070000000000000000000000000004A
:1046D00000010101010101010000000000000000D3
:1046E000003030000000000000000000806018046E
:1046F000006018060100000000E010080810E0004B
:10470000000F102020100F00001010F80000000013
:104710000020203F2020000000700808088870005A
:1047200000302824222130000030088888483000DA
:104730000018202020110E000000C02010F80000FA
:1047400000070424243F240000F808888808080093
:104750000019212020110E0000E0108888180000A8
:10476000000F112020110E0000380808C83808007A
:104770000000003F000000000070880808887000FA
:10478000001C222121221C0000E010080810E0007B
:104790000000312222110F00000000C0C000000004
:1047A0000000003030000000000000800000000029
:1047B0000000806000000000000080402010080021
:1047C00000010204081020004040404040404000EA
:1047D00004040404040404000008102040800000C5
:1047E0000020100804020100007048080808F000CA
:1047F0000000003036010000C030C828E810E0009A
:104800000718272423140B000000C038E000000024
:10481000203C23020227382008F88888887000008E
:10482000203F202020110E00C03008080808380062
:10483000071820202010080008F808080810E000D9
:10484000203F202020100F0008F88888E80810007A
:10485000203F20202320180008F88888E80810004E
:10486000203F200003000000C03008080838000086
:1048700007182020221E020008F808000008F80887
:10488000203F210101213F20000808F8080800000E
:104890000020203F2020000000000808F808080041
:1048A000C08080807F00000008F888C028180800B9
:1048B000203F20012638200008F8080000000000F2
:1048C000203F20202020300008F8F800F8F80800E9
:1048D000203F003F003F200008F830C00008F808E3
:1048E000203F200007183F00E01008080810E000F3
:1048F0000F10202020100F0008F808080808F0000A
:10490000203F210101010000E01008080810E0002C
:104910000F18242438504F0008F8888888887000C1
:10492000203F2000030C3020007088080808380061
:104930000038202121221C00180808F80808180057
:104940000000203F2000000008F808000008F808D8
:10495000001F202020201F000878880000C8380889
:10496000000007380E010000F80800F80008F80001
:10497000033C0700073C030008186880806818089B
:1049800020302C03032C30200838C800C838080019
:104990000000203F2000000010080808C838080068
:1049A0002038262120201800000000FE020202000C
:1049B0000000007F40404000000C30C000000000BC
:1049C000000000010638C00000020202FE000000E4
:1049D000004040407F00000000000402020204008A
:1049E00000000000000000000000000000000000C7
:1049F00080808080808080800002020400000000AF
:104A000000000000000000000000808080800000A6
:104A10000019242222223F2008F800808000000094
:104A2000003F112020110E00000000808080000057
:104A3000000E112020201100000000808088F80066
:104A4000000E112020103F20000080808080000098
:104A5000001F222222221300008080F088888818FC
:104A60000020203F20200000000080808080800007
:104A7000006B94949493600008F80080808000009C
:104A8000203F210000203F20008098980000000077
:104A90000020203F202000000000008098980000A7
:104AA00000C08080807F000008F8000080808000C7
:104AB000203F24022D302000000808F800000000EC
:104AC0000020203F202000008080808080808000A7
:104AD000203F20003F20003F808000808080000039
:104AE000203F210000203F200000808080800000C7
:104AF000001F202020201F008080008080000000F8
:104B000080FFA12020110E00000000808080800026
:104B1000000E112020A0FF80808080008080800017
:104B200020203F2120000100000080808080800044
:104B30000033242424241900008080E080800000B9
:104B40000000001F20200000808000000080800006
:104B5000001F202020103F20808080000080808067
:104B600000010E30080601008080008000808080F7
:104B70000F300C030C300F0000808000808080001C
:104B80000020312E0E312000808080000080808047
:104B900080818E70180601000080808080808000F7
:104BA0000021302C2221300000000000807C020215
:104BB00000000000003F404000000000FF00000037
:104BC00000000000FF0000000002027C80000000E6
:104BD0000040403F00000000000601010202040402
:104BE00000000000000000001060028C0000FE9237
:104BF00092929292FE00000004047E01407E4242A6
:104C00007E427E42427E40001060028C00FE929204
:104C100092929292FE00000004047E014448507F6C
:104C200040407F5048444000807000FF1008FE4222
:104C30004242FA424242FE00806018070810FF50CC
:104C4000484641424C40FF00100C055555D5057FA4
:104C50000555555505140C001010108AA96B352503
:104C600025ABE908101010001060028C201808C84D
:104C700038CF08082898000004047E01040201FFD0
:104C80004021060A112040000000FC242424FC25B9
:104C90002624FC242424040040308F80844C552595
:104CA0002525554C808080001010D0FF9014E4AF73
:104CB000A4A4A4AFE4040000040300FF00894B2A6D
:104CC0001A0E1A2A4B888000101090909090901025
:104CD00010FF101011161000002060203F1010105F
:104CE00000030C102040F800000000F8888C8A892E
:104CF000888888F800000000000000FF4444444415
:104D0000444444FF000000004044C4444444401074
:104D100010FF101010F00000103C131014B84030B9
:104D20000E014080403F000000002424242424FC85
:104D30002222222322000000020202020242827F7B
:104D400002020202020202004044C44444444010F1
:104D500010FF101010F00000103C131014B8403079
:104D60000E014080403F0000000022322AA6A262CD
:104D70002111098101000000004222130B42827EB2
:104D800002020A12234600002030AC63300088C8BB
:104D9000A8998E88A8C88800226722121280403005
:104DA0000F00003F4040710000F80122A0A2A222A3
:104DB000FE22AA3202FE000000FF0010130A4B2060
:104DC000170C133880FF0000008060F80704E4A48B
:104DD000A4BFA4A4E4040000010000FF40407F4AF7
:104DE0004A4A4A4A7F4040004042CC0000FE82923C
:104DF00092FE929282FE000000003F10887F001E0B
:104E00001212125E807F0000044444445F44C44494
:104E100044445F44C4040400000000000000FF009C
:104E200000081008070000000D0AE68C89E994AE1E
:104E3000E68EA7E588B6E8AFB4E6988EEFBC9AE6B2
:104E40008C89E4B88B4B4559312850413029E58F86
:104E5000AFE58887E68DA2E7BBA7E794B5E599A8FB
:104E6000E78AB6E680815C720A0000000D0AE58AD6
:104E70009FE883BDEFBC9A312EE5AE9AE697B6E582
:104E80008F91E980814448543131E6B8A9E6B9BF31
:104E9000E5BAA6E695B0E68DAE2020322EE68EA5C8
:104EA000E694B657694669E591BDE4BBA4E68EA7D2
:104EB000E588B64C45442020332E4448543131E631
:104EC00095B0E68DAE573235513634E5AD98E58272
:104ED000A82020342EE68C89E994AEE68EA7E588DA
:104EE000B6E7BBA7E794B5E599A85C720A00000095
:104EF0000D0A573235513634E5AD98E582A8E8AF52
:104F0000B4E6988EEFBC9AE6AF8F32E7A792E887B7
:104F1000AAE58AA8E5AD98E582A8E69C80E696B069
:104F20004448543131E695B0E68DAEE588B057324D
:104F300035513634E5A496E983A8466C617368E47C
:104F4000B8AD5C720A000000E8AEB0E5BD95202562
:104F5000643A20E697B6E997B4E688B33D256473D2
:104F60002C20E6B8A9E5BAA63D25642E2564E28486
:104F7000832C20E6B9BFE5BAA63D25642E2564251D
:104F80002552482C20E6A0A1E9AA8C3D3078253096
:104F900032580D0A000000000D0A0D0AE8AFBBE50B
:104FA0008F964448543131E68890E58A9F210D0A56
:104FB000E6B9BFE5BAA6E4B8BA25642E2564202573
:104FC00025524820EFBC8CE6B8A9E5BAA6E4B8BAE9
:104FD0002025642E2564E28483200D0A0000000051
:104FE0004C45445F524544004C45445F5055525037
:104FF0004C4500004C45445F57484954450000006B
:105000004C45445F424C5545000000004C45445F10
:105010005247424F464600004C45445F4359414E7B
:10502000000000004C45445F475245454E000000DB
:105030004C45445F59454C4C4F5700005C500008AC
:10504000000000206C00000078410008C8500008F3
:105050006C0000203C0C00008841000800A24A04BB
:105060000000000000000000010203040607080918
:1050700000000000010203040102030406070809FE
:10508000020406080000000000000000000000000C
:10509000000000000000000000000000E04F0008D9
:1050A000245000080050000830500008E84F000865
:1050B00018500008F44F00080C50000800000000D1
:0850C0000000000000000000E8
:0400000508000131BD
:00000001FF
